:1000000005308A00DB2D0000FF00030E8301A100F4
:100010000A08A0008A010408A2007708A300780853
:10002000A4007908A5007A08A600831383128C30F7
:100030008400801C1D288C182E2822088400230888
:10004000F7002408F8002508F9002608FA0020081F
:100050008A00210E8300FF0E7F0E09008A110A120A
:1000600039280A108A100A11820728340C34013406
:100070000634CC012830CB00AB0A2B08183C0318FF
:100080006C28AB0102304B07840083134C18831794
:10009000800A00083B3C03186C2802304B078400A0
:1000A00083134C188317800101304B07840083139E
:1000B0004C188317800A00083B3C03186C28013059
:1000C0004B07840083134C18831780014B0884006E
:1000D00083134C188317800A8C108A110A121D286A
:1000E0000634093409340634803480348034803452
:1000F0000034F43270366F3A611DA0123317313379
:100100009121201000008316851283128516831614
:100110000512831205168316811309128312941295
:10012000A71227088316870083122716270883162D
:1001300087008312A71127088316870001308312D6
:1001400094000030831694000108C73908388100F4
:10015000831290014830F80006389200F930831677
:10016000920007309C00050885000330F700F70B6C
:10017000B7281C0883120D1383169D01C03083120B
:100180008B0483168C141F149F101F159F111F13AF
:1001900083121F179F1383169F1783121F1400309B
:1001A000F8001F08C73978049F008A110A12EF2D42
:1001B0003F308400831300080319EC280130F80055
:1001C000F701F70BE128F80BE0284A30F700F70BAE
:1001D000E728EA28800BDE2808000808F039C70065
:1001E00045080F394704880007152711270883168B
:1001F0008700000083120711271127088316870044
:1002000083120800C308031D0729871008298714D3
:10021000A7102708831687008312C40E4408C50060
:10022000ED20C40E4408C500ED200D30F700F70B9B
:1002300017290800C830BF00D820F0308316880581
:1002400083128710A71027088316870083120711CF
:1002500027112708831687008312AD012D08023C61
:10026000031C3A290230BF00D8200330C500ED201E
:10027000AD0A2E290D30F700F70B3C290230C500DE
:10028000ED200D30F700F70B4329AD012D08023C9E
:10029000031C56292D083120AE00C3012E08C400CE
:1002A00002210230BF00D820AD0A46298A110A1265
:1002B000F82D831603178C170C140000000083120E
:1002C0008C08031980290D080313AD0003170F08CC
:1002D0000313AE0003170C080313AF000130C30073
:1002E0002F08C40002212D0803178D0003132E08C8
:1002F00003178F008D0A03198F0A03135929031757
:1003000003138A110A12062E83168C1002308312F0
:100310002D07840083132E18831780012D08840075
:1003200083132E188317800101302D078400831357
:100330002E188317800183168C1483128A110A12D7
:10034000112E01303F02C1004008023C031DAA29C2
:100350004030C10741088038C200C3014208C400D0
:10036000022108003008F8012F020318BA292F08CB
:10037000F700C629F7010830B100AF0DF70D3008BE
:1003800077020318F700F80DB10BBD2908003E08ED
:100390000C3A0319D229063A0319DA29073A031944
:1003A000E029E529C3010130C40002210230BF0069
:1003B000D820F1290130BF000230C000A121F1296D
:1003C0000130BF00C000A121F1293E081F3C031CE1
:1003D000EB290730BE050130C3003E08C4000221EE
:1003E000F129080078082D08AF006430B000B22170
:1003F0007708AD0078083030031D052AAE1C0C2AA2
:10040000AE190C2A2E1A2030082AAE112E122E14E4
:10041000F8077808BE00C7212D08AF000A30B000E9
:10042000B2217708AD0078083030031D1D2AAE19BF
:10043000212A2E1C212A2E1A2030F8077808BE0007
:10044000C7213030AD072D08BE00C72108003E0887
:100450000319972AC60042080319972AC6070318EA
:10046000382A7F30C602031C972A0319972A3C2A90
:100470008130C6070318972A4608F700F801F901EA
:10048000FA013F08CA00CA174008C9004108C8005D
:100490001830C600C701481C652A4508FA07031C26
:1004A000572AF90A031D572AF80A0319C7174408DF
:1004B000F907031C5E2AF80A0319C7174308C0008E
:1004C000C0174008F8070318C717C70DF80CF90C38
:1004D000FA0CCA0CC90CC80C0310C60B4A2A01300E
:1004E000F7070318972AF81B7C2ACA0DFA0DF90D95
:1004F000F80DF7030319972ACA1F8D2AFA0A031D5C
:100500008D2AF90A031D8D2AF80A031D8D2AF80C7D
:10051000F90CFA0CF70A0319972A3F08C700430899
:10052000C706C71F952AF8179B2AF8139B2AF701BD
:10053000F801F901FA010800AE01AD01AF012F0881
:100540001F3C031CB52A1F151F19A42A83161E0859
:100550008312AD071E0803181E0FAE071030F700F8
:10056000F70BB02A0000AF0A9F2A2E0CFA002D0CC0
:10057000F900FA0CF90CFA0CF90CFA0CF90CFA0C5B
:10058000F90C0730FA057908F8007A08F9007908BB
:10059000FA007808AD007A08AE008E30F7002E0819
:1005A000F8002D08F900FA01F808031DE12A79087E
:1005B000F800F9010830F702F808031DE12AF701F5
:1005C000E92A0310F81BE82AF90DF80DF703E12AD0
:1005D000F8137030C1009830C0002C30BF007E305E
:1005E000BE007A08C5007908C4007808C3007708FF
:1005F000C20027227708AD007808AE007908AF0066
:100600007A08B000B2010408B1003210831B321422
:1006100083143008B6002F08B5002E08B4002D084A
:10062000B300CD30BA002C30B9001330B800873099
:10063000B70080308318B806BD01BE013408BC0085
:100640003808BC0633080319092CBB00F70037082B
:100650000319122CBB020319AE2B031C6C2B380898
:10066000C100C1173908C0003A08BF00BE0103101D
:10067000C10CC00CBF0CBE0CBB0B362BBC1F432BDC
:100680003D14262C3D103B103D163630840083135C
:100690003B2C3D12BC1B562B3B1C612BC10CC00CD0
:1006A000BF0CBE0CF70A0319212C612BC11B642B54
:1006B0000310BE0DBF0DC00DC10DF7030319212C92
:1006C000562B3D17CE2B3D133408BC00BC1F6A2BA4
:1006D000C1171A2CC1131A2C3708BB00F7003308B6
:1006E000BB023408C100C1173508C0003608BF007E
:1006F000BE010310C10CC00CBF0CBE0CBB0B782B91
:10070000BC1F852BBD14262CBD103B10BD163A30E6
:10071000840083133B2CBD12BC1B982B3B1CA32BCA
:10072000C10CC00CBF0CBE0CF70A0319212CA32B63
:10073000C11BA62B0310BE0DBF0DC00DC10DF703CD
:100740000319212C982BBD17CE2BBD133808BC00E4
:10075000BC1FAC2BC1171A2CC1131A2C3808C100AE
:10076000C1173908C0003A08BF00BC1FBB2BC1131A
:100770003D15262C3D11BE013B10363084008313FD
:100780003B2CBC1BE42B3408BC003B1CCE2BC10C07
:10079000C00CBF0CBE0CF70A0319212CBE1FDF2BA7
:1007A000BF0A031DDF2BC00A031DDF2BC10A031D77
:1007B000DF2BC10CC00CBF0CF70A0319212C3D1B09
:1007C000632BBD1BA52B032C8030C106C11FEC2B56
:1007D000262C3808BC00F92B3408BC00C108031DC6
:1007E000F92BC008031DF92BBF08031DF92BF701D6
:1007F0001A2CC11B032C0310BE0DBF0DC00DC10D63
:10080000F70BF92B212CBC1F072CC1171A2CC11375
:100810001A2C3708F7003808C1003908C0003A0818
:10082000BF001A2C3308F7003408C1003508C00097
:100830003608BF004108F8004008F9003F08FA00F8
:10084000592CF701F801F901FA01592CBE01BF0931
:10085000C009C109BE09BE0A031D342CBF0A031D0D
:10086000342CC00A0319C10A3D18422BBD18842B31
:100870003D19BA2BE92B0008BF07031C452CC00A01
:10088000031D452CC10A03193B1484030008C0074B
:10089000031C4D2CC10A03193B1484030008801F5C
:1008A000803AC10703183B143D1A492BBD1A8B2B04
:1008B000C12B310884008313321883178A110A125E
:1008C0003E2E831603178C170C140000000003182B
:1008D000902C83120C087F390313B20003170D0804
:1008E0000313B30003170F080313B4003208BE004C
:1008F000C721330803178D000313340803178F0033
:1009000083168C170C140000000083120313B10B24
:100910008A2C8D2C83160317902CAF2C831603176B
:1009200083120C0D0E0D7F390313B20003170D084F
:100930000313B30003170F080313B4003208BE00FB
:10094000C721330803178D000313340803178F00E2
:100950008D0A03198F0A03100313B10B612C0800D1
:10096000F701F801F901FA01C601C701C801C9017F
:1009700045084404430442040319EE2C2030CA0005
:100980000310BE0DBF0DC00DC10DC60DC70DC80DA6
:10099000C90D45084902031DD72C44084802031D10
:1009A000D72C43084702031DD72C42084602031CDC
:1009B000E82C4208C6024308031C430FC702440840
:1009C000031C440FC8024508031C450FC902031449
:1009D000F70DF80DF90DFA0DCA0BC02C4630840046
:1009E000831308000408B6003508B8000319112D58
:1009F0003408C1003308C0003208BF003108BE000F
:100A0000C501C4012030C3008230C20027227A0809
:100A1000B4007908B3007808B2007708B100B80BC9
:100A2000F82C3408C1003308C0003208BF00310878
:100A3000BE003E08B63CBE00FA013F08C200BF1728
:100A40000310BF0CC00CC10CFA0CF90CF80CF70C1D
:100A5000BE0B202DC21F372DF709F809F909FA0935
:100A6000F70A0319F80A0319F90A0319FA0A7A08A6
:100A7000B4007908B3007808B2007708B100B41F59
:100A80004E2DB603B616B109B209B309B409B10ABD
:100A90000319B20A0319B30A0319B40A3B30BD00A3
:100AA0009A30BC00CA30BB00BA010A30B800350821
:100AB0000319B60A3408C1003308C0003208BF0069
:100AC0003108BE003D08C5003C08C4003B08C30017
:100AD0003A08C200B0240008B100840A0008B2003D
:100AE000840A0008B300840A0008B400FD308407BB
:100AF000F708031D8E2D350A380203198E2D36088E
:100B00000319902D0F3938020319882D0318C02DB1
:100B1000B61BC02D361B902D2030BC2D2030B605C5
:100B2000B61E9E2DB6123508031DB6037708B60013
:100B30002D30BE00C7213608F700B601350838024F
:100B4000031DAC2D7708B6002E30BE00C721360835
:100B5000F7002030B60500303030B61EBC2DB6127E
:100B60003508031DB6037708B6002D30BE00C72137
:100B70003608F700B6013030F7077708BE00C72106
:100B80003D08C1003C08C0003B08BF003A08BE0059
:100B9000C501C401C3010A30C200B0247A08BD00F7
:100BA0007908BC007808BB007708BA00B80B5A2D4A
:100BB0008A110A125D2E840183131F308305831668
:100BC000861383128617AB0183161F149F141F15FB
:100BD0009F1107309C00FF308312A70083288316E3
:100BE00085128312851683160512831205161A299B
:100BF000C3014830C40002210230BF00D820703049
:100C000003178D0000308F0003135929C3010330EF
:100C1000C40002210230BF00D820AE012830AD0050
:100C200084290230AD009630BF00D820AD0B132EC2
:100C30002C082A020319382E2A08AC000930BF00FC
:100C40000130C000A1212808AD001130AE00F22112
:100C50003A30BE00C7212908AD000130AE00F221B4
:100C60003A30BE00C7212A08AD000130AE00F221A3
:100C70000130BF000230C000A1219C2A7708AD00DE
:100C80007808AE007908AF007A08B0007930031711
:100C90008D0000308F00031009300313B100612470
:100CA000023084003008B4002F08B3002E08B200D0
:100CB0002D08B1000130B500F22C803003178D00F3
:100CC00000308F00031004300313B1006124112E93
:020CD0006300BF
:02400E003A3F37
:00000001FF
